:02000000352E9B
:10000800FF00030E83018316A4000A08A3008A01D7
:1000180070088312A4007B08A3007C08A2007D0856
:10002800A1000B1C6828851A26284130FC00EE30F8
:10003800FD00FD0B1D28FC0B1D2800000515851E65
:100048002328E401051A45284130FC00EE30FD0064
:10005800FD0B2C28FC0B2C2800000515051E31284B
:100068000130E4000230FB004530FC00A930FD00FF
:10007800FD0B3C28FC0B3C28FB0B3C280000000037
:100088000511851968284130FC00EE30FD00FD0B94
:100098004B28FC0B4B280000E2014130FC00EE30FD
:1000A800FD00FD0B5528FC0B55280000E20A6208EC
:1000B800143C03186428DF010130DD0005156628AB
:1000C8000130DF00851D51280B102408F00023089B
:1000D800FB002208FC002108FD00831623088A0083
:0A00E800240E8300FF0E7F0E0900B6
:1000F2008316BF03BF033F08003C03188528BF03D4
:100102000000000000007C28000000000000000049
:0401120000000800E1
:1001160083120313F8010830FC00700DF80D740803
:10012600F80203189828F8070310F00DFC0B902826
:020136000800BF
:100138008316A0018030F00080303E067002031D57
:10014800A7283D0820020318B4284130FC00EE30EF
:10015800FD00FD0BAD28FC0BAD280000A00A9E2871
:0201680008008D
:10016A007408F8027508031C750FF9027608031C57
:10017A00760FFA027708031C770FFB02F30D07309C
:10018A00FC00730DF80DF90DFA0DFB0D7408731CC4
:10019A00DC28F8027508031C750FF9027608031C9F
:1001AA00760FFA027708031C770FFB02E928F80793
:1001BA0075080318750FF90776080318760FFA07FA
:1001CA0077080318770FFB07F30DFC0BC628720D8F
:1001DA00F80DF90DFA0DFB0D7408731C0229F802CB
:1001EA007508031C750FF9027608031C760FFA02CC
:1001FA007708031C770FFB020F29F8077508031805
:10020A00750FF90776080318760FFA0777080318A7
:10021A00770FFB07F20D0730FC00720DF80DF90D90
:10022A00FA0DFB0D7408721C2829F8027508031CC4
:10023A00750FF9027608031C760FFA027708031C79
:10024A00770FFB023529F80775080318750FF907A8
:10025A0076080318760FFA0777080318770FFB0753
:10026A00F20DFC0B1229710DF80DF90DFA0DFB0DAB
:10027A007408721C4E29F8027508031C750FF902DE
:10028A007608031C760FFA027708031C770FFB0225
:10029A005B29F80775080318750FF907760803181C
:1002AA00760FFA0777080318770FFB07F10D073067
:1002BA00FC00710DF80DF90DFA0DFB0D7408711C97
:1002CA007429F8027508031C750FF9027608031CD5
:1002DA00760FFA027708031C770FFB028129F807C9
:1002EA0075080318750FF90776080318760FFA07C9
:1002FA0077080318770FFB07F10DFC0B5E29700DC9
:10030A00F80DF90DFA0DFB0D7408711C9A29F80203
:10031A007508031C750FF9027608031C760FFA029A
:10032A007708031C770FFB02A729F807750803183B
:10033A00750FF90776080318760FFA077708031876
:10034A00770FFB07F00D0730FC00700DF80DF90D63
:10035A00FA0DFB0D7408701CC029F8027508031CFD
:10036A00750FF9027608031C760FFA027708031C48
:10037A00770FFB02CD29F80775080318750FF907DF
:10038A0076080318760FFA0777080318770FFB0722
:10039A00F00DFC0BAA297018E0297408F8077508F3
:1003AA000318750FF90776080318760FFA07770806
:0803BA000318770FFB07080090
:1003C20001308316BE0083126B088316BD068312AA
:1003D2006F0884006B08003A0319F229650880044B
:1003E200F429680880056A088316BF007920BD09D0
:1003F2003E080319162A3E083D05F000031D052A92
:10040200831265088004082A83126808800583160F
:10041200BE0D3E10023083126A028316BF0079209D
:100422000000000000000000F92983126B08003A66
:1004320003191E2A68088005202A650880046A08B4
:080442008316BF0079200800B9
:10044A00FB09FA09F909F809F80A0319F90A03195B
:08045A00FA0A0319FB0A08006D
:0E046200A530FD00FD0B332A0000000008004D
:0C047000831626088A0025088200080078
:10047C0083120313FC01F71BFC0AFD01FB01FA01BB
:10048C00F901F80173087204710470040319D22A7B
:10049C0073087706A000A01BFD09F71F602AF4095A
:1004AC00F509F609F709F40A0319F50A0319F60A0E
:1004BC000319F70AF31F6D2AF009F109F209F30980
:1004CC00F00A0319F10A0319F20A0319F30A730863
:1004DC007704A000A01B8E2AB520FC1BAB2AFD1FA5
:1004EC00D22AF009F109F209F309F00A0319F10A09
:1004FC000319F20A0319F30AF809F909FA09FB09B5
:10050C00F80A0319F90A0319FA0A0319FB0AD22A81
:10051C00F71FA52AF31B9F2A7308FB007208FA0029
:10052C007108F9007008F800F301F201F101F00113
:10053C00752AF301F201F101F001F00A0034F3091C
:10054C00F209F109F009FC17722AF80A0319F90AE1
:10055C000319FA0A0319FB0A74087802031D752A99
:10056C0075087902031D752A76087A02031D752A0F
:10057C0077087B02031D752AFB01FA01F901F801CA
:10058C00F00A0319F10A0319F20A0319F30AF31F0B
:10059C00752AA0012016FF34A0017C1CD62A252226
:0405AC00003E080005
:0C05B0001030FD00FD0BDA2A00000800EE
:1005BC00831203132230FC00F801F901FA01FB014C
:1005CC00FC030319142B0310FB0CFA0CF90CF80C9C
:1005DC00F30CF20CF10CF00C031CE62AFC030319CF
:1005EC00062B7408F80775080318750FF9077608B9
:1005FC000318760FFA0777080318770FFB07EA2A18
:10060C007408F80775080318750FF90776080318AE
:0E061C00760FFA0777080318770FFB07080020
:10062A000A308316BD00E1210D30BD00E12108002A
:10063A00A0308312F0000F30F100F201F30108003C
:10064A00831238088316BC006430F4003A08F000BC
:10065A008B200A30F4008B207808F0003030F00745
:10066A0083163C088400700880008312380A8316B7
:10067A00BC000A30F4003A08F0008B200A30F4007B
:10068A008B207808F0003030F00783163C0884008D
:10069A00700880000230831238078316BC000A30C3
:1006AA00F4003A08F0008B207808F0003030F007A8
:1006BA0083163C08840070088000BB013B08023C9A
:1006CA00031C762B3B088312380784000008831624
:1006DA00BD00E1210130BD000030BE009C20BB0AF4
:0A06EA00632B04308312850608001C
:0E06F4001930FD00FD0B7C2B000000000800FB
:1007020083163A089B009C131C141A08F000080078
:0407120000000800DB
:1007160083162908F1000130F00071080319972BA0
:10072600F00D7010FF3E912B7008AB00F009280801
:1007360084007008800584177008800531222B0814
:10074600800484137A232B080005AA002A08003A9D
:10075600013003190030AA0031222A08F0000800EF
:1007660083169C1CB82B0000B32B28089B00290875
:100776009A009C131C150B08F0008B1355309D0036
:10078600AA309D009C14F01BCA2B8B13CB2B8B1706
:040796001C1108002A
:10079A00DC2B8312F101F201F52B3C30F100003021
:1007AA00F200F52B5830F1000230F200F52B003040
:1007BA0083162906031DE32B003028060319CE2BC6
:1007CA0000302906031DEB2B063028060319D22B0D
:1007DA0000302906031DF32B0C3028060319D72BEA
:1007EA008312E2018030F000803072067002031D2D
:1007FA00002C710862020318152C6408031D152CBD
:10080A000630FB001330FC00AD30FD00FD0B0B2C55
:10081A00FC0B0B2CFB0B0B2C00000000E20AF72B45
:02082A000800C4
:10082C0083162908F1000130F00071080319222CFD
:10083C00F00D7010FF3E1C2C7008AD00F009700814
:10084C00AC0028088400700880058417AB012B08C5
:10085C00073C031C472C2B08F0002A08F1007008F9
:10086C0003193C2CF10CF113FF3E362C2C0880059F
:10087C00711C422C2D0880047A232D088004AB0AAD
:0A088C002D2C8413D822D822080076
:100896008316BA0181237008A8007008FF3A031D69
:1008A600552CA8018312051501308316BD000030B2
:1008B600BE009C20A9010630290203186F2C2908C6
:1008C600563E84000008BD00E1210130BD00003025
:1008D600BE009C20A90A5E2C1523A9010830290216
:1008E6000318822C29084D3E84000008BD00E12132
:1008F6000130BD000030BE009C20A90A712C2808DA
:10090600BA0025231523A9010E3029020318982CB5
:1009160029083A3E84000008BD00E1210130BD00EF
:100926000030BE009C20A90A872C83126308831618
:10093600A900063083126307F100F2010318F20AD8
:100946008030F000803072067002031DAD2C7108F5
:10095600831629020318BD2C83162908253E840018
:100966000008BD00E1210130BD000030BE009C2022
:10097600A90A9C2C15232808003C0318E52C0230F4
:10098600AA002808013EF100F2010318F20A80309D
:100996007206F00080307002031DD32C2A08710203
:1009A600031CE52C2A08BA0081237008BA00252307
:1009B600F8308316BD00E1214330BD00E121152347
:0609C600AA0AC42C08007F
:1009CC0038228A110A128000840AA50A0319A60A81
:0809DC00F003031DE62C0800E6
:1009E40083162908F1000130F00071080319FE2C68
:1009F400F00D7010FF3EF82C7008AD007009AC00CB
:100A040028088400AB01AA012A08073C031C2A2DEC
:100A14002C08800584172C08800589232D08800460
:100A2400892384132D080005F0000319262D2A08B4
:100A3400F1000130F00071080319242DF00D70103D
:100A4400FF3E1E2D7008AB04D822D822AA0A062D18
:060A54002B08F000080071
:100A5A00831628088312EF0083162908F000013054
:100A6A00F200700803193D2DF20D7210FF3E372D6A
:100A7A0072088312E7007209E60083162A08F10059
:100A8A000130F000710803194E2DF00D7010FF3E71
:100A9A00482D70088312E500F0097008E8008030DC
:100AAA008316280784007208800470088005831260
:100ABA00EB0183162F080319642D8312EB098312A5
:100ACA0084136B08003A03196D2D680880056F2D91
:100ADA00650880041D23E830F4000330F500F601B0
:100AEA00F701DE2270088316B0007108B10072089F
:100AFA00B2007308B3002B08F0002C08F1002D088F
:100B0A00F2002E08F300F00DF10DF20DF30D701046
:100B1A00F00DF10DF20DF30D70100A30F400F5012D
:100B2A00F601F701DE2270088316B4007108B500D9
:100B3A007208B6007308B7007008F4007108F5006F
:100B4A007208F6007308F7003008F0003108F10067
:100B5A003208F2003308F3003E2270088316B80008
:100B6A007108B9007108F400F501740875040319D5
:100B7A00C12D0230F000080038088312EA008316FB
:100B8A003408F4003508F5003608F6003708F7008F
:100B9A003008F0003108F1003208F2003308F3009F
:100BAA003E227808F0007908F1007A08F2007B0802
:100BBA00F30070088316B0007108B1007208B20021
:100BCA007308B3003408F5003508F6003608F70054
:100BDA003708F800F80CF70CF60CF50CF813781B2C
:100BEA00F81780307806F400803073067402031D0B
:100BFA00082E72087702031D082E71087602031D5B
:100C0A00082E7008750203180C2E8312EA0A831242
:100C1A006A08F100F10CF1137108E900073071025A
:0E0C2A0003181A2E0130F0000800F001080037
:100C38008312E201033062020318342E05150230D4
:100C48008316BD000030BE009C20831205110230BF
:100C58008316BD000030BE009C208312E20A1E2EBF
:020C6800080082
:100C6A009C27FF308316A70007308312990039307A
:100C7A00831685009F0101308312E400DF01DE0143
:100C8A00DD011C268316BA01812370088312E00055
:100C9A007008FF3A031D522EE00105308316A800A2
:100CAA00A9010130AA008030AB002530AC00AD01AB
:100CBA00AE01AF012D2583127008E100851A6A2E54
:100CCA008316A70183120515632E051A722E0630A4
:100CDA008316A700831205156A2E85197A2E0C3001
:100CEA008316A70083120515722E803083162706F5
:100CFA00F0008030003A7002031C892E0130A800EF
:100D0A002708A900B3231C2601308316BA008123C1
:100D1A0070088312E3007008FF3A031D952EE30161
:100D2A008B178B15383083169600831239086002A8
:100D3A0003180E2F6408003A031D0E2F0530831680
:100D4A00A800A9018B230530A800A901CC30AA006C
:100D5A0016240530A800A9014430AA0016248B17CE
:100D6A000A30BD000030BE009C200530A800A90151
:100D7A008B230530A800A901CC30AA0016240A301A
:100D8A00BD000030BE009C200530A800A901BE307D
:100D9A00AA0016240530A800A901F22470088312BB
:100DAA00EC00ED0105308316A800A901F2247008B1
:100DBA00F200F10183126C087107F300720803183C
:100DCA00013E6D07F4007308EC007408ED00730827
:100DDA00F0007408F100F10CF00CF1137008EE0049
:100DEA008B13023060078316A8007008A900B3238A
:100DFA008312E00A8316A801831260088316A900E9
:100E0A00B3238B171C2663088316A800A901CD23D8
:100E1A00232F39086002031C232F6408003A031D9C
:100E2A00232F0130DE00051514308316BD00003073
:100E3A00BE009C20831205110130E4005F080319EB
:100E4A002C2F8B114B248312DF0105118B155D08A2
:100E5A00013A031D542F8B118316A101A2010230FE
:100E6A0083123907F100F2010318F20A83162208E5
:100E7A007202031D422F21087102031C4C2F210804
:100E8A00A800A901B323A10A0319A20A342F8312C5
:100E9A00DD010130E4000511E001E3018B15413069
:100EAA00FC00EE30FD00FD0B582FFC0B582F000004
:040EBA009A2E5E2FDF
:100F38002530840038308312F00064308316A50011
:080F48000730A600E6240800B2
:100EC800313420345334653463342034313420349D
:100ED8004D3469346E3420343134303420344D3458
:060EE80069346E34003491
:020EEE00493485
:020EF000F034DC
:100EF200533461346D3470346C3469346E34673415
:0E0F02002034543469346D3465343D34003489
:080F1000303430343034003479
:100F1800533461346D3470346C34653473343D3417
:020F2800003493
:0E0F2A00523461346A344C346F34673400340E
:02400E00D40FCD
:00000001FF
